:1000000018308A00342C0000FF00030E8301A10089
:100010000A08A0008A010408A2007708A300780853
:10002000A4007908A5007A08A6007B08A70083131E
:1000300083128C308400001C1F280C1832282208E0
:1000400084002308F7002408F8002508F900260892
:10005000FA002708FB0020088A00210E8300FF0E0B
:100060007F0E09008A110A1241280A108A100A110B
:10007000820700340034103430348A3400340034C1
:100080002D34061D452806114628061564000C105F
:100090008A110A121F28871087162130F700F70BE4
:1000A0004F2800348C1A5628640052288C1E56287B
:1000B0001A088316B9008312981C64281A0883163C
:1000C000B90083121812181683163908F800831223
:1000D00000342908073C031D722807300C1E6E28C7
:1000E0009900B12805308316A7002708063C03199C
:1000F000B0282708053C031DAA282930A90083122F
:100100006F088316A600043083120C1E8528990000
:100110006F080C1E892899008316A80183126F08A6
:10012000831628020318A428290884000008AA00BE
:1001300083120C1E99289900831629088400000850
:10014000A606A90AA80A8E28260883120C1EA6282D
:10015000990083168312522078088316A700752809
:10016000831200349030A9000130AA002930AB007E
:10017000831681138312861DC0280230AC00C2286A
:100180000130AC000430EF0069200034C830840036
:1001900000080319D8280630F800F701F70BCE281D
:1001A000F80BCD287B30F700F70BD428800BCB2839
:1001B00000349130A9000230EF0069202A08F700CE
:1001C000F7080319F828013077020319FE280230D6
:1001D0007702031904290330770203190A2906302C
:1001E00077020319102907307702031916291D29F0
:1001F000813083169900263098001F2940308316DD
:100200009900263098001F29203083169900263047
:1002100098001F29153083169900263098001F2951
:100220000A3083169900263098001F29043083165F
:100230009900263098001F29831283161F29023047
:10024000C8008312C6208A150A12F52EF701F8019C
:1002500083163A0803103B18F707F70CF80CBB1885
:10026000F707F70CF80C3B19F707F70CF80CBB195C
:10027000F707F70CF80C3B1AF707F70CF80CBB1A4A
:10028000F707F70CF80C3B1BF707F70CF80CBB1B38
:10029000F707F70CF80C831200349230A9006F08AE
:1002A000413C03196A290130AA00FE017E083F3C47
:1002B000031C692902307E07293E84007E088316CC
:1002C000BA000530BB008312262178088000FE0AA0
:1002D0005629A229FE017E083F3C031C86290130D5
:1002E0007E07293E840000088316A1007E08BA001C
:1002F0000530BB00831226217808831621020319DA
:10030000832983128629FE0A83126B297E083F3CCB
:10031000031C8C2901308D290030AA00FE017E08C3
:100320003F3C031CA22902307E07293E84007E0840
:100330008316BA000530BB0083122621780880009E
:10034000FE0A8F294230EF0069208A150A12FD2E1D
:100350009530A9000508AA000608AB000708AC0004
:10036000053083169F0083121F083839C1389F005B
:100370000030F8001F08C73978049F00A630F70046
:10038000F70BC02900001F151F19C4291E08AD0056
:100390000830F8001F08C73978049F00A630F7001E
:1003A000F70BD02900001F151F19D4291E08AE0015
:1003B0000630EF00692000346F08073C031DF32965
:1003C0002A088316850083122B0883168600831261
:1003D0002C088316870083122D0885002E088600BE
:1003E0002F088700A8218A150A12052F2A088316CC
:1003F000A0002B30A100FE01023083126F027E02AA
:100400000318302A83162008A00AA2002108A10A96
:1004100084000008A3002208831203178D008F01B7
:10042000831603132308831203178C0083168C137F
:100430000C15831203130B08F7008B138316031795
:1004400055308D00AA308D008C148C18252A0C1183
:100450007708831203138B04FE0A8316FC29831288
:100460000730A9000130EF0069208A150A12152F04
:100470002A088316A0002B30A10083122B08EF005E
:10048000FE016F087E020318592A83162108A10A6B
:1004900084002008A00AA300831203178D008F0197
:1004A00083168C130C1483120C088000FE0A0313AD
:1004B000412AE330A9000230EF0769208A150A12A9
:1004C0001D2FE530A9000130AA000230EF0069209D
:1004D0008A150A12252FE730A9004630AA000230FB
:1004E000EF0069208A150A122D2F87120034803000
:1004F0008316870581308704D93086050616DB30E0
:1005000085051B3085040515851686148312871111
:1005100007124B20752287142130F700F70B8E2A23
:100520004B20752287142130F700F70B952A2808F5
:10053000FF3E0318AE2A013EAF2A83164608C700C5
:10054000F501F4014708F6001F3C031DAC2A643096
:10055000C8008312C62083168312AE2A00340A1004
:100560008A140A1182079D2A2A08FE007E08E039B3
:10057000A8007E088316C600831277220730A900E0
:100580000130EF0069208A150A12352F7E102A08E3
:100590000139003A0319D02A6F08023C03197E146E
:1005A00000307E1801308316A000A10083124B207A
:1005B00007110C3097000030F800043892007730B3
:1005C00083169200A1080319ED2A3C30831295008E
:1005D0001708CF399700F32A83162030831295002D
:1005E0001708CF3997004B2004308316A000AF3096
:1005F000C8008312C6208316A00BF72A0730831287
:10060000A9000130EF0069208A150A123D2F071159
:10061000970197014B200730A9000130EF006920B6
:100620008A150A12452F76081F3C031D382B8316A6
:10063000CB014B08053C031C362B83128715031096
:100640008316C90C0318282B831207122A2B831632
:10065000831207162130F700F70B2C2B871121305E
:10066000F700F70B312B8316CB0A192B6D2C831255
:1006700083164908E03E03186D2C203E8312742C2B
:10068000071287158711071287158711071287151B
:10069000871107128715871107128715871107120F
:1006A0008715871183166D2C07168715871107127A
:1006B000871587110712871587110712871587116C
:1006C00007128715871107128715871183166D2C5E
:1006D00007128715871107168715871107128715C7
:1006E00087110712871587110712871587110712BF
:1006F0008715871183166D2C071687158711071626
:10070000871587110712871587110712871587111B
:1007100007128715871107128715871183166D2C0D
:100720000712871587110712871587110716871576
:10073000871107128715871107128715871107126E
:100740008715871183166D2C0716871587110712D9
:1007500087158711071687158711071287158711C7
:1007600007128715871107128715871183166D2CBD
:100770000712871587110716871587110716871522
:10078000871107128715871107128715871107121E
:100790008715871183166D2C071687158711071685
:1007A0008715871107168715871107128715871177
:1007B00007128715871107128715871183166D2C6D
:1007C00007128715871107128715871107128715DA
:1007D00087110716871587110712871587110712CA
:1007E0008715871183166D2C071687158711071239
:1007F0008715871107128715871107168715871127
:1008000007128715871107128715871183166D2C1C
:100810000716871587110716871587110712871581
:100820008711071687158711071287158711071279
:100830008715871183166D2C0712871587110716E8
:1008400087158711071687158711071687158711D2
:1008500007128715871107128715871183166D2CCC
:10086000071687158711071687158711071687152D
:100870008711071287158711071687158711071229
:100880008715871183166D2C07128715871107129C
:100890008715871107128715871107168715871186
:1008A00007168715871107128715871183166D2C78
:1008B00007168715871107168715871107168715DD
:1008C00087110716871587110716871587110712D5
:1008D0008715871183166D2C831600000000000019
:1008E00000000000831200340A108A100A158207E3
:1008F000402B542B682B7C2B902BA42BB82BCC2B70
:10090000E02BF42B6C2C082C6C2C6C2C1C2C6C2CE1
:100910006C2C6C2C6C2C6C2C6C2C6C2C6C2C302C53
:10092000442C6C2C6C2C6C2C6C2C6C2C6C2C582C43
:1009300076081F3C031DD42C871507162130F700BD
:10094000F70BA02C87112130F700F70BA52C83168D
:10095000CB014B080D3C031CC72C831287150310D9
:100960008316CA0CC90C0318B92C83120712BB2CAE
:100970008316831207162130F700F70BBD2C871161
:100980002130F700F70BC22C8316CB0AA92C831257
:10099000871507162130F700F70BCC2C8711213073
:1009A000F700F70BD12CF32C871507168711831648
:1009B000CB014B080D3C031CEF2C83128715031051
:1009C0008316CA0CC90C0318E92C83120712EB2CEE
:1009D00083168312071687118316CB0AD92C83122C
:1009E0008715071687110330F700F70BF52C003435
:1009F00083164608C9008312132383164808CA00C9
:100A00004708C900831298240034831645087502EC
:100A1000031C102D031D182D74084402031C182DEF
:100A200045081F3C03182D2D75081F3C031C2D2D58
:100A300045081F3C031C222D7608C600831277222E
:100A40002C2D8316C6013F30C800FF30C70083122B
:100A5000F8242030F500F401831675084502031CC4
:100A6000402D031D372D440874020318402D063015
:100A7000C90083121323F40A0319F50A83162D2DD6
:100A80008312003483163A08C90083121323831695
:100A90003B08C8008312C6208316BC080319552DD5
:100AA0003C08C90083121323831601307407BD006C
:100AB0007508BE000318BE0A3E08C5003D08C40004
:100AC00083120525003483162108FD3E0318842D6A
:100AD000033E83129D2D09308316A1002030C500EE
:100AE000C401831205258316842D0B308316A100C3
:100AF000842D1F308316A1002030C500C40183124D
:100B000005258316842D83162108C900831213231B
:100B1000831621081F3C0319962D0830BA000430B3
:100B2000BB00BC01831242259A2D83160430C800F5
:100B30008312C6208A150A12A82B0A148A100A15D5
:100B400082076B2D752D792D83162108FD3E031824
:100B5000D22D033E8312D62D8316C901831213238F
:100B60003F308316CA00FF30C90083129824093031
:100B70008316C9008312132306308316C80083121C
:100B8000C6208316A1080319D22D0B308316C90085
:100B90008312132306308316C8008312C6208316DF
:100BA000D22D831683128A150A12382C0A148A1041
:100BB0000A158207AC2DC52DAC2D83164208C9003D
:100BC00083121323831607164308C40076081F3CBC
:100BD000031D0C2EC50145080F3C031C0B2E831270
:100BE00087150000071AF62D0310F72D031483163E
:100BF00044088400840A800C8403800C2130F700B0
:100C0000F70B002E831287112130F700F70B062E09
:100C10008316C50AEB2D252EC50145080F3C031C84
:100C2000252E831287150000071A182E0310192E7F
:100C30000314831644088400840A800C8403800C07
:100C4000831287118316C50A0D2E440884000130D3
:100C500084070310800C8403800C4408840000087F
:100C6000F700840A00083F39FA00770884038000FF
:100C7000840A7A0880000330F700F70B3D2E071234
:100C8000831200348316AE012D082E020318642E41
:100C90002B08FA002A08AA0A0319AB0AAF007A083F
:100CA000B000C5002F08C4008312052583162E0846
:100CB0002C07AF000430C2002F08C3008312DD25CB
:100CC00002308316AE07442E831200348316310897
:100CD000B40010307602F33E0318A52E0D3E8312A9
:100CE000D62E08308316B500B600A52E0430831624
:100CF000B5001830B600A52E0D308316B5000830AB
:100D0000B600A52E08308316B5001830B600A52E03
:100D100003308316B5000830B600A52E08308316C0
:100D2000B500B600A52E14308316B5000830B60005
:100D3000A52E08308316B500B600A52E0430831604
:100D4000B5001830B600A52E83163008C5002F0850
:100D5000C400831205258316B30132083302031839
:100D6000D22E01303307340784000008B80034085D
:100D7000330784000008B9003808BA000230C60002
:100D80003808C8003908C7008312F82483163608CB
:100D9000BA003508BB00BC0183124225023083161D
:100DA000B307AD2E83128A150A12E2280A108A149C
:100DB0000A158207712E762EA42EA42EA42E7C2E28
:100DC000822E8E2E932E992E9E2EA42E882E831642
:100DD00039080739BE007608123C031D192FF83078
:100DE000B9053F30BA05BD013E083D020318192F71
:100DF0003A08FA003908B90A0319BA0AC2007A088F
:100E0000C300C5004208C4008312052504308316C0
:100E1000C200BF30C3008312DD2502308316C60036
:100E20004008C8003F08C7008312F8248316BD0A93
:100E3000F42EBD013C083D020318422F3A08FA0087
:100E40003908B90A0319BA0AC2007A08C300C500F2
:100E50004208C4008312052583163B08BB0ABB0A5F
:100E60008400840A0008C30084030008C200023022
:100E7000C6004308C8004208C7008312F82483163E
:100E8000BD0A1A2F7608123C031D762F3A081F3C24
:100E900003184D2F0430C1004F2F0830C1003E0809
:100EA000BC0741083C020318762F3A08FA003908BB
:100EB000B90A0319BA0AC2007A08C300C500420879
:100EC000C4008312052504308316C200BF30C3005E
:100ED0008312DD2502308316C6004008C8003F0893
:100EE000C7008312F8248316BC0A512F83120034E2
:100EF0008316BD0101303C023D020318A22F3B08BE
:100F0000BB0ABB0A8400840A0008BF0084030008EF
:100F1000BE000230C6003F08C8003E08C70083126A
:100F2000F824013074078316BE007508BF0003184B
:100F3000BF0A3F08C5003E08C4008312052583167A
:100F4000BD0A7A2F3B088400840A0008BF0084038E
:100F50000008BE000230C6003F08C8003E08C700B7
:100F60008312F824003483162108FD3E0318D02F85
:100F7000033E8312D72F20308316C500C40183128D
:100F8000052509308316C900831213238316D02F39
:100F90000B308316C900831213238316D02F8316B8
:100FA0000630C8008312C6208A150A12882C0A143B
:100FB0008A140A158207C12FC82FBB2F2808FF3EAD
:100FC0000318EC2F013EF12F7E088316A0008A152E
:100FD0008312372B8A11EC2F871107128A150A12F8
:100FE000A32C0A148A140A158207E42F00308C1AE5
:060FF0000130F80000349E
:101000008316B5013108B6000310B20C2F0807395A
:10101000F70030080039FA007708083CB4003408BB
:101020003202031815283208B40012307602FE3E50
:1010300003182C28023E8312C92806308316B700F5
:101040000830B8002C2802308316B7001830B800DA
:101050001730B5002C28831630081F3C031867286A
:10106000FF3A031D37282F08033C03186728300870
:10107000C5002F08C4008A11831205258A1583161E
:10108000B30132083302031866283608B60AB60AD6
:101090008400840A0008BA0084030008B900023002
:1010A000C6003A08C8003908C7008A118312F8241C
:1010B0008A1508308316BA000630BB00BC018A11BD
:1010C000831242258A158316B30A4128C5283008A1
:1010D000BA002F08B9003108BB003408BC008A11DF
:1010E0008312E7268A1583163808BA003708BB0032
:1010F0003508BC008A11831242258A1583163408EC
:10110000B2020310340DF700B6070830B3003308FD
:101110003202031CA8287508BA007408B900360802
:10112000BB000830BC008A118312E7268A1583169B
:101130003808BA003708BB003508BC008A11831292
:1011400042258A1510308316B6070830B307872862
:101150000730B205B2080319C5287508BA0074082B
:10116000B9003608BB003208BC008A118312E7269A
:101170008A1583163808BA003708BB003508BC004A
:101180008A11831242258A15831683128A150A1240
:10119000EF280A108A100A1182071D282328103010
:1011A0007602F03E0318D02A103ED12A83162C086E
:1011B000B0002B08AF002D08B1002E08B2008A1134
:1011C0008312662E8A15D02A83162C08B0002B08AD
:1011D000AF002D08B1002E08B20083120028D02ADB
:1011E00083162C08B0002B08AF002D08B1002E0884
:1011F000B2003108B4000310B20C0130B500083061
:10120000B6000E30B3003008C5002F08C4008A11A4
:10121000831205258A1583162F080139F700300837
:101220000039FA0077087A04031937293408B40A18
:10123000B40A8400840A0008B80084030008B700D8
:101240000230C6003808C8003708C7008A11831268
:10125000F8248A1583163608BA003508BB0033080F
:10126000BC008A11831242258A158316B203320804
:10127000013C031883293408B40AB40A8400840AA0
:101280000008B80084030008B7000230C600380820
:10129000C8003708C7008A118312F8248A15013064
:1012A00074078316B7007508B8000318B80A380821
:1012B000C5003708C4008A11831205258A158316D4
:1012C0003408B40AB40A8400840A0008B80084030D
:1012D0000008B7000230C6003808C8003708C70049
:1012E0008A118312F8248A1583163608BA00350845
:1012F000BB003308BC008A11831242258A150230D4
:101300008316B2023729B2080319A6293408B40A91
:10131000B40A8400840A0008B80084030008B700F7
:101320000230C6003808C8003708C7008A11831287
:10133000F8248A1583163608BA003508BB0033082E
:10134000BC008A11831242258A1583168312D02A83
:1013500083162C08B0002B08AF002D08B1002E0812
:10136000B2003108B7000310B20C2F080339B500E2
:10137000043CB40032020318BF293208B400013023
:10138000B8001830B9001730B6003008C5002F0873
:10139000C4008A11831205258A158316B50803191E
:1013A000EB293108BB003408BC008A11831278276E
:1013B0008A1583163908BA003808BB003608BC0005
:1013C0008A11831242258A1583163408B20203104B
:1013D000340DF700B7070430B30033083202031CA2
:1013E0000A2A3708BB000430BC008A118312782710
:1013F0008A1583163908BA003808BB003608BC00C5
:101400008A11831242258A1508308316B7070430E3
:10141000B307ED290330B2050319252A3208033931
:10142000BA003708BB003A08BC008A11831278273B
:101430008A1583163908BA003808BB003608BC0084
:101440008A11831242258A1583168312D02A8316A5
:101450002C08B0002B08AF002D08B1002E08B200F8
:101460003108B3000310B20C3008FA002F08AF0A9D
:101470000319B00ABA007A08BB00C5003A08C400D4
:101480008A11831205258A158316B2080319CE2AFC
:10149000B8013308B30AB30A8400840A0008FA00CA
:1014A00084030008B4007A08B5003808B80A183C6C
:1014B000031CBB2A0230C6003508C8003408C70028
:1014C0008A118312F8248A1508308316C9008A11FC
:1014D000831213238A15A630F700F70B6D2A00003C
:1014E0000E308316C9008A11831213238A15043023
:1014F0008316C200B630C3008A118312DD258A1517
:10150000831634083602031DBA2A35083702031D34
:10151000BA2A3808BA000330BB008A118312262188
:101520008A1578088316B800B901380839020318FB
:10153000B92A0230C6003508C8003408C7008A112D
:101540008312F8248A1508308316C9008A11831281
:1015500013238A15A630F700F70BAC2A00000E30D3
:101560008316C9008A11831213238A158316B90AB8
:10157000952ABB2A552AB2033008FA002F08AF0A71
:101580000319B00ABA007A08BB00C5003A08C400C3
:101590008A11831205258A15442A83168312D02ABC
:1015A00000340A108A140A118207D628D628E428A3
:1015B000E428F028D628D628D628D628D628D62813
:1015C000A829D628D628D02A272A83162108FD3E06
:1015D00003182C2B033E8312302B20308316AB00D4
:1015E0000730AA00A530AC000230AD008A1183128A
:1015F00042268A1509308316C9008A1183121323E3
:101600008A1508308316C8008A118312C6208A15ED
:10161000FF308316A5040F30A6042030AC0007303D
:10162000AB00A530AD000230AE008312CF20831690
:10163000A10803192C2B0B308316C9008A118312C1
:1016400013238A1508308316C8008A118312C62016
:101650008A1583162C2B831683128A150A123F2CA7
:101660000A148A140A118207ED2A1B2BED2A103066
:101670007602F23E03188A2C0E3E8D2C831620082B
:10168000A1002108F700F708831203194C2B013041
:1016900077020319502B552B02308316A100572BCC
:1016A00003308316A100572B83128316A101210852
:1016B000C9008A11831213238A153F308316CA008A
:1016C000FF30C9008A11831298248A158316A10855
:1016D000031D782BA2012208063C031C782B063040
:1016E000C9008A11831213238A158316A20A6B2B51
:1016F0000130C9008A11831213238A15073083161B
:10170000C9008A11831213238A1508308316C90071
:101710008A11831213238A1508308316C8008A1190
:101720008312C6208A1501308316C9008A118312DC
:1017300013238A1507308316C9008A1183121323D5
:101740008A158A2C83162008A1008A118312632D22
:101750008A158A2C09308316C9008A118312132333
:101760008A151E308316C8008A118312C6208A1576
:101770008A2C83162008A1002108F700F70883129D
:101780000319C72B013077020319CB2BD02B09305B
:101790008316A300D12B0B308316A300D12B831209
:1017A0008316C9018A11831213238A153F308316C9
:1017B000CA00FF30C9008A11831298248A15831643
:1017C000A2012208063C031CEE2B0630C9008A1138
:1017D000831213238A158316A20AE12B2108023CE7
:1017E0000319082C2308C9008A11831213238A15B0
:1017F00018308316C9008A11831213238A15053005
:101800008316C8008A118312C6208A15312C8316CC
:101810000130C9008A11831213238A1507308316F9
:10182000C9008A11831213238A1508308316C90050
:101830008A11831213238A150D308316C8008A116A
:101840008312C6208A1501308316C9008A118312BB
:1018500013238A1507308316C9008A1183121323B4
:101860008A158A2C83162008A1008A118312A42DC0
:101870008A158A2C83162008A1008312E52A8A2C57
:1018800083162008A1000230A2001730A3002030E8
:10189000C500C4018A11831205258A158316210803
:1018A000F700F708831203195A2C01307702031945
:1018B000652C712C09308316C9008A1183121323F9
:1018C0008A1508308316A100772C0B308316C900C7
:1018D0008A11831213238A1508308316A100772CEE
:1018E00083121F308316A1000830A200A301210833
:1018F000BA002208BB002308BC008A1183124225CB
:101900008A158A2C83162008A1008A118312B32F0E
:101910008A158A2C8A110A12EA2F0A108A100A15CF
:1019200082073E2B3E2BA22BA22BAA2BB92BB92B25
:101930003A2C3E2BB92BB92B402C322C822C2A0866
:10194000FE008A11DE2F8A150730A9000130EF0052
:101950008A1169208A158A150A124C2F2808FF3E21
:101960000318C02C013EC52C83162608AC002508A0
:10197000AB002908AD002A08AE008312CF20C02C8E
:10198000871107128A150A12EB2C0A108A100A1501
:101990008207B42C8316A30183122C088316A2009D
:1019A00083122B088316A10083122A088316A00035
:1019B000043083126F02FE0083162308A800220859
:1019C000A7002108A6002008A5002D30A9007E0848
:1019D000AA008312AE2C0730A9000130EF008A1153
:1019E00069208A158A150A12522F2808FF3E03180B
:1019F000092D013E0E2D83162508AB002408AA00F0
:101A00002808AC002908AD008A11831242268A15E5
:101A1000092D871107128A150A12352D0A148A100A
:101A20000A158207FB2C8316A30183122C08831648
:101A3000A20083122B088316A10083122A088316A2
:101A4000A00083122D08EF0083162308A7002208A8
:101A5000A6002108A5002008A4002D30A8008312AC
:101A60006F088316A9008312F52CC430A900043036
:101A7000EF078A1169208A158A150A12582F8316D2
:101A8000AE0110307602F23E0318932D0E3E831203
:101A9000C12D08308316AC00AD00932D083083169D
:101AA000AC00AD00932D0D308316AC000830AD00B6
:101AB000932D04308316AC001830AD00932D023006
:101AC0008316AC001830AD001730AE00932D0830EF
:101AD0008316AC001830AD00932D06308316AC0091
:101AE0000830AD00932D08308316AC00AD00932D67
:101AF00014308316AC000830AD00932D14308316DB
:101B0000AC000830AD00932D04308316AC001830C3
:101B1000AD00932D01308316AC001830AD001730A6
:101B2000AE00932D83162808C5002708C4008A112B
:101B3000831205258A158316AB012A082B02031888
:101B4000BD2D2B08290784000008AF000330C60014
:101B5000C8012F08C7008A118312F8248A1583163A
:101B60002D08BA002C08BB002E08BC008A11831275
:101B700042258A158316AB0A9D2D83128A150A12F7
:101B8000E42D0A148A100A158207492D592D4E2D6D
:101B90005F2D922D532D672D732D782D7E2D842D45
:101BA0008A2D6D2D732D2808FF3E0318E52D013E6B
:101BB000EA2D83162408A8002308A7002508A900F9
:101BC0002608AA0083123F2DE52D871107128A15DA
:101BD0000A12052E0A148A100A158207D92D2B081D
:101BE0008316A10083122A088316A00003308312F3
:101BF0006F02FE0083162108A4002008A3002C30E9
:101C0000A5007E08A6008312D32D0730A90001305D
:101C1000EF008A1169208A158A150A125E2F28089A
:101C2000FF3E0318462E013E4B2E83162308A700C5
:101C30002208A6002408A8002508A900AA0129084E
:101C40002A020318442E2708FA002608A60A0319B8
:101C5000A70AAD007A08AE00C5002D08C4008A119D
:101C6000831205258A1505308316C200AB30C300E8
:101C70008A118312DD258A1583162A082807840015
:101C80002B088000AA0A1F2E8312462E87110712E6
:101C90008A150A12672E0A108A140A158207152E51
:101CA0002B088316A10083122A088316A000831232
:101CB0002C08EF0083162108A3002008A2002C3076
:101CC000A40083126F088316A50083120F2EE23042
:101CD000A9000330EF078A1169208A158A150A12B4
:101CE000642F8A114B208A15D030A900AA01AB01BC
:101CF000AC01AD010530EF008A1169208A158A1503
:101D00000A126A2F8A1175228A15D030A900013073
:101D1000AA00AB01AC01AD010530EF008A116920CA
:101D20008A158A150A12702F0130FD008316A20150
:101D30002930A300A208031DE62E8A118312522027
:101D40008A157808FE007E08043C0319AD2E8A111E
:101D500052208A157808FE00A32E8A1152208A1577
:101D60007808EF008316A100A00183126F08831684
:101D700020020318CD2E2308A4008A1183125220BA
:101D80008A158316240884007808800023088400BC
:101D90000008A106A30AA00AB52E8A1183125220B8
:101DA0008A1578088316A106031DDF2E0130A200D4
:101DB000063083120C1EDA2E9900E42E83160530AD
:101DC00083120C1EE12E990083169A2E8312290885
:101DD000103C031DEF2E8A11B2208A15722F29089C
:101DE000113C031DF72E8A11D9288A15722F290854
:101DF000123C031DFF2E8A114D298A15722F2908C6
:101E0000143C031D072F8A11DC298A15722F29081B
:101E1000153C031D0F2F8A11A8218A15722F29083E
:101E2000173C031D172F8A11F6298A15722F2908CE
:101E3000183C031D1F2F8A11382A8A15722F290872
:101E40001A3C031D272F8A11612A8A15722F29082F
:101E50001B3C031D2F2F8A116B2A8A15722F29080C
:101E6000413C031D372F8A11B42A8A15722F290885
:101E7000403C031D3F2F8A11C62A8A15722F29085C
:101E8000473C031D472F8A11072B8A15722F2908FB
:101E9000433C031D4D2F9F2C722F2908423C031DEC
:101EA000532FCA2C722F2908443C031D592F132D80
:101EB000722F2908453C031D5F2FEF2D722F290833
:101EC000463C031D652F502E722F2908503C031DE0
:101ED0006B2F712E722F2908513C031D712F822EFA
:101EE000722FFD017D08F8008A150A169D2CCC3052
:101EF000840000080319812F7F2F00000000800B51
:101F00007D2F8A150A129A2F83164B1464008312B0
:101F1000071E9B2F640083164A08CA03003A031D5C
:101F2000962F4B1083129B2F9A2F8316FF30CC00D5
:101F30008312772F882F003083164B180130F8005A
:101F4000831200340408F8000830F7000718A62FA1
:101F50008316BA01F717BE2FF713BE2F0310831293
:101F6000071803148316BA0C7717BE2F7713F70BD5
:101F7000AE2F780884003A08F800D52F023084008C
:101F80000030F71B5530F800F80BC42F840BC02F1E
:101F9000AB30F71B2E30F800F80BCC2F0000000000
:101FA000F71BAC2F771BB62FAE2F83128A110A16A0
:101FB000902908300C1EDA2F9900831636088312F8
:101FC0000C1EE02F9900003403300C1EE52F990001
:101FD0008316260883120C1EEB2F99008316260801
:101FE0008312EE00003429080C1EF42F99002908F2
:041FF000EE060034C5
:102000008316420DC300C30DC30DF830C305071678
:10201000FF30CA000A128A15831284270A168A1111
:102020008316C501C40145087102031C2528031D40
:102030001D2844087002031C25280230F700F70B06
:102040001F28C40A0319C50A13288312871583168B
:10205000C501C40145087102031C3D28031D342835
:1020600044087002031C3D280630F700F70B3628A1
:102070000000C40A0319C50A2A288312071A422835
:102080000310432803148316C60DC70DC80D07128D
:10209000831207128316420B53280310BE0D031C34
:1020A0005328071668284208023C031D5E280310C7
:1020B000BE0DBF0D031C5E28071668284208033CAE
:1020C000031D68280310BE0DBF0DC00D03180716B1
:1020D000831287118316C501C40145087102031CD0
:1020E0008028031D772844087002031C80280630CE
:1020F000F700F70B79280000C40A0319C50A6D28F8
:102100000716C30B252807164608F7004708F800EE
:102110004808F9004908FA00831200340710083013
:10212000F800000000000000F817A728F813831635
:10213000B70C831203180714031C07107817A7287D
:102140007813F80B972800000000000007140230F5
:10215000F7008401840BAA28F70BA928AD3084006E
:10216000840BB02800000000F81B9628781BA028DC
:102170008A110A16282AFF308316B400B500B6006B
:10218000B701CA010A128A15831284270A168A1116
:10219000F8080319EB282808FF3E0318EB28013E36
:1021A000F6288316C101C0014030BF00BE010230D5
:1021B000C2008312002078081F39FA007708F8005F
:1021C0007A08F9008316B701B6017908B5007808D6
:1021D000B4008312EB2883163408F7003508F800A2
:1021E0003608F9003708FA00831200340A108A1002
:1021F0000A118207D128FF308316B000B100B20067
:10220000B301CA010A128A15831284270A168A1199
:10221000F80803195E292808FF3E03185E29013ECD
:10222000652A83162C08B5002B08B4002C08B700CB
:102230002B08B600FF30B800B9003608F7003708A1
:102240001F39FA003608BA007A08C038BB00BC0152
:10225000BD013D08C1003C08C0003B08BF00360876
:10226000BE000230C200831200208316CA010A1287
:102270008A15831284270A168A11F808031951292E
:102280008316C101C0014030BF00BE010230C20050
:102290008312002077088316B80078081F39B90028
:1022A000831283163808F8003908F900B301B20127
:1022B0007908B1007808B00083125E298316AF0850
:1022C00003193D2A341034183D2ACA010A128A150E
:1022D000831284270A168A11F808031971298316B4
:1022E0003D2AB5308316B6003714B7108610831216
:1022F0008614831607147C1C82293608840001305A
:102300008000BD29B718BD296400831207189A29D7
:10231000831636088400B9000A128A158312A22F88
:102320000A168A1183163908840078088000B714C9
:10233000BC2983120A12F6270A16F8080319AC29D9
:102340000A1252200A167808023C031DAB29831694
:10235000B71437108312BB298316CA010A128A15D3
:10236000831284270A168A11F8080319BB298316D9
:10237000B7143710831283168229003037180130C2
:10238000F800F8080319392A3508F70001307702F8
:1023900083120319CC292E2A01308316B6000A12A3
:1023A0008A158312D9270A168A11B5308316B6000A
:1023B0003714B710B718182ACA010A128A158312DF
:1023C00084270A168A11F8080319E8298316182A9F
:1023D0000A12F6270A16F8080319162A8316360871
:1023E000B8000A12831252200A1683163808840095
:1023F00078088000360884000008083C031D0D2A78
:102400003608B8000A12831252200A1683163808BA
:10241000840078088000B714152A36088400000864
:10242000023C031D152AB714371083128316DA29CC
:10243000003037180130F800F80803192A2A7C10F8
:102440003508B600861407103608B70083128E28A8
:102450002D2A83167C1434148312372A83163508E8
:10246000B6000A128A158312D9270A168A113B2A46
:1024700083163414831283166329300F462A310FD2
:10248000462A320F462AB3080319502A300F5B2A16
:10249000310F5B2AB208031D5B2AB308031D5B2AB8
:1024A0008312BB207A088316B3007908B20078083B
:1024B000B1007708B0003008F7003108F8003208A2
:1024C000F9003308FA00831200340A108A140A1142
:1024D000820711290A124B200A1687150A12752243
:1024E0000A161030F700F70B732A00008711FF302F
:1024F0008316CA000A128A15831284270A168A11C3
:102500008316AE01AD01AC01AB01AF018312FB201C
:102510000A124B200A1687150A1275220A16103065
:10252000F700F70B912A000087118316C101C00143
:102530004030BF00BE010230C20083120020780884
:102540001F39FA007708F8007A08F900003483167A
:10255000A901AA010230F1007130F000FF30CA0079
:102560000A128A15831284270A168A11F808031999
:102570001B2B8316C101C0011030BF00BE01023009
:10258000C20083120020831607168312071AC62A78
:102590008316AA01A90183128715F3010130F20005
:1025A000071ADB2AF20A0319F30A720873040319E3
:1025B000DB2A6400D02A071AE62AF20A0319F30A72
:1025C000720873040319E62A6400DB2A8312071ECB
:1025D000F82A8316A90A0319AA0A29082A04031942
:1025E000F82A12306400FF3E031DF22A0000E62A9A
:1025F00083128711720873040319152B8316290897
:102600002A04031D052B8312152B2A0CF100290C1B
:10261000F000F10CF00CF10CF00CF10CF00CF10CE2
:10262000F00C0730F1051A2B83120230F1007130E3
:10263000F0008316831283162908F8002A08F9008F
:102640008312003483160511831205158316851233
:102650008312851683168610831286142808FF3E7F
:1026600003183F2B013E602B6A226A228316A801C1
:10267000A7017908A6007808A50083123F2BA7229E
:10268000FF308316CA000A128A15831284270A169D
:102690008A11F808031D532B8316A801FF30A700E9
:1026A000A600A500831283162508F7002608F80067
:1026B0002708F9002808FA0083128A110A166A2BE3
:1026C0000A148A140A118207342BA0308316A4003E
:1026D0008312222B7A088316A3007908A2007808B7
:1026E000A1007708A000D0308312A9008316CA0188
:1026F0000A128A15831284270A168A11F808031908
:10270000832B0030842B0130AA0083162408A40AEE
:10271000840000088312AB0083162408A40A8400F6
:1027200000088312AC00831624088400000883127A
:10273000AD000530EF000A1269200A168A150A1644
:10274000D02B8316A801FF30A700A600A500CA0160
:102750000A128A15831284270A168A11F808031DA3
:10276000E12B8715A630F700F70BB42B000087117B
:102770002808FF3E0318D82B013EEE2B8316C1011B
:10278000C0014030BF00BE010230C20083120020F1
:1027900078081F39FA007708F8007A08F9008316DC
:1027A000A801A7017908A6007808A5008312D82BF4
:1027B000FF308316CA000A128A15831284270A166C
:1027C0008A1183162508F7002608F8002708F90063
:1027D0002808FA0083128A110A16F82B0A148A14A0
:1027E0000A118207BE2BA0308316A4008312A12BEE
:1027F0007A088316A3007908A2007808A100770858
:10280000A000D0308312A9008316CA010A128A15CB
:10281000831284270A168A11F8080319112C003034
:10282000122C0130AA0083162408A40A8400000890
:102830008312AB0083162408A40A840000088312C4
:10284000AC0083162408840000088312AD00053014
:10285000EF000A1269200A168A150A16D82B831669
:102860002514A030A40083126F08053C031D442CDE
:102870002D080139003A031D412C83162510432CE5
:1028800083128316251483128316A90183122C0840
:102890008316A80083122B088316A70083122A0828
:1028A0008316A600003025180130AA002908AE00C2
:1028B0002808AD002708AC002608AB002A08AF00A6
:1028C0008312FB207A088316A3007908A2007808F7
:1028D000A1007708A000D0308312A9008316CA0196
:1028E0000A128A15831284270A168A11F808031916
:1028F0007B2C00307C2C0130AA0083162408A40A0B
:10290000840000088312AB0083162408A40A840004
:1029100000088312AC008316240884000008831288
:10292000AD000530EF000A1269200A168A150A1652
:10293000E02BFF308316CA000A128A1583128427FF
:102940000A168A11F8080319CF2C2808FF3E03182D
:10295000CF2C013EEF2C8316C101C001FF30BF0018
:10296000BE000230C200831200208316C101C001E4
:102970004030BF00BE010230C20083120020780840
:102980001F39FA007708F8007A08F9008316A801C1
:10299000A7017908A6007808A5008312CF2CFF3084
:1029A0008316CA000A128A15831284270A168A110E
:1029B000F808031DE22C8316A801FF30A700A6002B
:1029C000A500831283162508F7002608F8002708BB
:1029D000F9002808FA0083128A110A16052F0A1036
:1029E0008A100A158207AB2C6E080C1EF52C990074
:1029F0000A1252200A167808063C031DF82C0034EF
:102A000084011F308305073083169F0040309900F2
:102A100026309800903083129800A001A101103058
:102A2000A2003030A3008A30A400A501A6012D30F9
:102A3000A70040308316990026309800903083120A
:102A40009800403083169900263098009030831209
:102A500098004030831699002630980090308312F9
:102A600098000F30F70007308101813084000008A2
:102A7000F0390738800064000008F03977048000DE
:102A800099256400DF26412D63008C1A492D6400CE
:102A9000452D8C1E492D1A088316A0008312981C00
:102AA000572D1A088316A0008312181218168316C1
:102AB0002008F800831200342808073C031D652D08
:102AC00007300C1E612D9900982D0530FC007C0804
:102AD000063C0319982D7C08053C031D942D2830D5
:102AE000FE006E08F60004300C1E742D99006E086E
:102AF0000C1E782D9900FD016E087D020318902DA3
:102B00007E08840000088316A00083120C1E862D08
:102B100099007E0884000008F606FE0AFD0A7C2D56
:102B200076080C1E912D990045257808FC00672D2C
:102B30000034B130A8000130EE005C250034F20111
:102B40002830F300F208031DDA2D45257808EF0040
:102B50006F08043C0319B02D45257808EF00A82D17
:102B600045257808EE006E08F100F0016E0870024D
:102B70000318C82D7308F4004525740884007808EC
:102B80008000730884000008F106F30AF00AB62DED
:102B900045257808F106F108031DD52D0130F20016
:102BA00006300C1ED12D9900D92D05300C1ED62DC6
:102BB0009900A22D00347C0803178D007D088F003A
:102BC00083168C170C140000000083120E08FA0004
:102BD0000C08F8000E08F900031300347D08143CBB
:102BE0000318F62D7D08163C03181F2E7C080317CA
:102BF0008D007D088F0083160313200883120317AE
:102C00008C00831603132108831203178E0083168A
:102C10008C170C15831203130B08F8008B13831603
:102C2000031755308D00AA308D008C140000000071
:102C30008C18182E0C117808831203138B0400349F
:102C40001F30AA052A08F0002908EF006F08033991
:102C5000F400FC30EF05F301740873020318492EE9
:102C60007008FD006F08FC00DB257908F200780889
:102C7000F1007008FD006F08FC0072088316A100C7
:102C80007108A0008312EE25EF0A0319F00AF30A77
:102C90002C2E2B30F5000330F3006E08730203185E
:102CA000812E750884000008F100840A0008F200F3
:102CB000F50AF50AF008031D702E6F08033C031C8B
:102CC000702E03106F0DF900700DFA007908203E88
:102CD0008400840A720880008403710880007B2EBF
:102CE0007008FD006F08FC0072088316A1007108CF
:102CF000A0008312EE25EF0A0319F00A0230F30751
:102D00004D2E6F080339F400F4080319AB2EF008B8
:102D1000031D8E2E6F08033C0318AB2E7408043C71
:102D20000319AB2E7008FD006F08FC00DB25790845
:102D3000F2007808F1007008FD006F08FC007208CE
:102D40008316A1007108A0008312EE25F40AEF0A91
:102D50000319F00A8E2E0730A8000130EE005C2522
:102D60000034EF016F08033C031CCD2E03106F0DE0
:102D7000F700203E8400840A0008F3008403000862
:102D8000F200FD016F08FC0073088316A1007208B1
:102D9000A0008312EE25EF0AB22ECD2E0034E430CF
:102DA000A8002030A9000230EE005C25003428087D
:102DB000A900FF30A8000230EE005C2500349F25FA
:102DC0002808313C031DE62E9925F92E2808323CAF
:102DD000031DEC2E2026F92E2808333C031DF22E6D
:102DE000B126F92E2808193C031DF82ECF26F92EFE
:042DF000D7260034AE
:102E0000A0308316A4008312992C7A088316A3009D
:102E10007908A2007808A1007708A000D0308312BA
:102E2000A9008316CA010A128A15831284270A167A
:102E30008A11F80803191E2F00301F2F0130AA0035
:102E400083162408A40A840000088312AB008316AA
:102E50002408A40A840000088312AC008316240806
:102E6000840000088312AD000530EF000A126920CB
:102E70000A168A150A16E82BA0308316A4008312BE
:102E8000BB207A088316A3007908A2007808A10065
:102E90007708A000D0308312A9008316CA010A1255
:102EA0008A15831284270A168A11F80803195A2FE3
:102EB00000305B2F0130AA0083162408A40A840086
:102EC00000088312AB0083162408A40A84000008BB
:102ED0008312AC0083162408840000088312AD001E
:102EE0000530EF000A1269200A168A150A16F02B1F
:102EF0008316A901FF30CA000A128A15831284279B
:102F00000A168A11F8080319922F8316C101C0010D
:102F1000BF01BE010130C200831200207708831672
:102F2000A900831283162908F8008312003483163F
:102F30002C08AD002030AE00AF01B0013008C10058
:102F40002F08C0002E08BF002D08BE000230C200AE
:102F5000831200208316C101C0014030BF00BE01B2
:102F60000230C2008312002078088316AF00770871
:102F7000AE002F08FA01F800831200348316AA016C
:102F8000FF30CA000A128A15831284270A168A1192
:102F9000F8080319DB2F2808FF3E0318DB2F013E3A
:102FA000E22F83162808AC0083129727780883162F
:102FB000AA008312DB2F83162A08F80083128A15D1
:102FC0000A1659290A148A140A158207D12F2908CA
:102FD000AA00FF30A9000230EF000A1269200A1689
:062FE0008A150A16302CD0
:1030000029308316A20083122B088316A100831295
:103010002A088316A00083122C088316A40003300C
:103020002407A500A6000A128312E4270A168316B5
:1030300022088400E03080000A128312F3270A1667
:1030400083162208840083122A0880000A12F327BC
:103050000A1683162208840083122B0880000A12A5
:10306000F3270A1683162208A5002108A7002008C6
:10307000A600FF30CA000A12831284270A16F80835
:103080000319642883162608F70027080F39FA0069
:103090002608A9007A084038AA00AB01AC012C0828
:1030A000C1002B08C0002A08BF002608BE0002305D
:1030B000C2008A11831200208A158A1178278A1586
:1030C00078088316A8008312FF308316CA000A12FC
:1030D000831284270A16F808031D7228FF3083160E
:1030E000A800831283162808F800250884007808B1
:1030F00080000A128312F3270A1601308316A300F8
:1031000024082302031896282208A5008A11831296
:1031100078278A15831625088400780880000A120B
:103120008312F3270A168316A30A80288A118312B2
:10313000F4248A158A150A16F72B2B088316A20089
:1031400083122A088316A1000330A00083126F089F
:1031500083162002031803292208FA002108A10A75
:103160000319A20AA3007A08A400293020078400CA
:103170000008A5002408A7002308A6002508A80029
:10318000FF30CA000A12831284270A16F8080319AE
:10319000002983162608F70027080F39FA002608A9
:1031A000A9007A085038AA00AB01AC012C08C10074
:1031B0002B08C0002A08BF002608BE000230C2004B
:1031C0008A11831200208A15FF308316CA000A1262
:1031D000831284270A1683162808A9006030AA00E3
:1031E000AB01AC012C08C1002B08C0002A08BF00AD
:1031F0002808BE000230C2008A11831200208A15FE
:103200008316A00AA62807308312A9000130EF0018
:103210000A128A1169200A168A158A150A16FD2BC8
:1032200029308316A20083122B088316A100831273
:103230002A088316A00083122C088316A4000330EA
:103240002407A500A6000A128312E4270A16831693
:1032500022088400E23080000A128312F3270A1643
:1032600083162208840083122A0880000A12F3279A
:103270000A1683162208840083122B0880000A1283
:10328000F3270A168316A3012408230203186629CC
:103290002208A5002108FA002008A00A0319A10AA3
:1032A000A6007A08A700A9002608A8008A118312A0
:1032B000BE2F8A15831625088400780880000A121C
:1032C0008312F3270A168316A30A44298A1183124C
:1032D000F4248A158A150A16032CFF308316CA00B7
:1032E0000A12831284270A16F8080319BB29280832
:1032F000FF3E0318BB29013EBE2983162308A70001
:103300002508A8002608A900AA0129082A020318EE
:10331000B9292A082707AB00AC008A118312972726
:103320008A15831628082A0784000008AB00AC0021
:10333000FF30CA000A12831284270A16F8080319FC
:10334000B62983162C08AD003030AE00AF01B001B5
:103350003008C1002F08C0002E08BF002C08BE0096
:103360000230C2008A11831200208A158316AA0A2D
:1033700085298312BB298A150A16D9290A148A10AD
:103380000A1182077D292B088316A10083122A08BF
:103390008316A000033083126F028316A200210857
:1033A000A4002008A3002C30A5002208A600831248
:1033B0006D290730A9000130EF000A128A11692037
:1033C0000A168A158A150A16092CFF308316CA00B8
:1033D0000A12831284270A16F8080319412A2808BA
:1033E000FF3E0318412A013E442A83162608AC00FA
:1033F0002508AB002908AD002A08AE002B08B00054
:103400002C08B1000830B200B3013308C100320803
:10341000C0002C08BF002B08BE000330C2008A1178
:10342000831200208A158316C1010930C000BF0134
:10343000BE010330C2008A11831200208A15831650
:10344000AF012E082F0203183F2A2D08AD0AAD0A3E
:10345000B000C1010930C000BF01BE010330C2008D
:103460008A11831200208A15831630088400770899
:103470008000840A780880000230AF07212A831276
:10348000412A8A150A166B2A0A108A140A11820721
:10349000F5298316A40183122C088316A300831236
:1034A0002B088316A20083122A088316A100831218
:1034B0002D08EF0083162408A8002308A70022087F
:1034C000A6002108A5002D30A90083126F088316DD
:1034D000AA008312E529C430A9000430EF070A12BC
:1034E0008A1169200A168A158A150A160F2CFF30D0
:1034F0008316CA000A12831284270A16F8080319D1
:10350000CE2A2808FF3E0318CE2A013ED12A831670
:103510002708AD002608AC002A08AE002B08AF0033
:103520002C08B1002D08B2000830B300B4013408F3
:10353000C1003308C0002D08BF002C08BE000330B6
:10354000C2008A11831200208A158316B0012F0849
:1035500030020318CC2A2E08AE0AAE0A8400840A70
:103560000008FA0084030008B1007A08B2000A30AB
:10357000B300B4013408C1003308C0003208BF00F2
:103580003108BE000330C2008A11831200208A1560
:1035900002308316B007A72A8312CE2A8A150A168C
:1035A000F72A0A108A140A118207872A8316A401AF
:1035B00083122C088316A30083122B088316A20003
:1035C00083122A088316A100043083126F02831627
:1035D000A5002408A9002308A8002208A7002108A4
:1035E000A6002D30AA002508AB008312772A0730E9
:1035F000A9000130EF000A128A1169200A168A1503
:103600008A150A16152C2A308316A00097308312CB
:10361000A90083162008A1008A118312A7228A1507
:10362000831621088400840A7908800084037808BE
:10363000800003308312EF000A128A1169200A16F3
:103640008A158A150A161B2C2A308316A0008312AD
:103650002C08EF00831620088400840A0008A200CA
:1036600084030008A1002208A4002108A3002C3034
:10367000A50083126F088316A600E6308312A90006
:103680000330EF070A128A1169200A168A158A1573
:103690000A16212C2A308316A00020088400840AF0
:1036A0000008A20084030008A100033083126F0207
:1036B0008316A3002208A5002108A4002C30A60030
:1036C0002308A70007308312A9000130EF000A1277
:1036D0008A1169200A168A158A150A16272C83165C
:1036E000A0012008033C031CC12BA2012008A1005B
:1036F0000310200DF700A300230A0A128A11831277
:1037000035200A168A15FA00831623080A128A1130
:10371000831235200A168A158316A4007A08A5009C
:103720002108831203178D008316031322088312C6
:1037300003178F00831603132408831203178C00CA
:10374000831603132508831203178E0083168C1724
:103750000C15831203130B08F8008B138316031741
:1037600055308D00AA308D008C14000000008C189C
:10377000B72B0C117808831203138B048316A00A4D
:10378000712B8A01831282018A150A162D2CFE08DC
:10379000031D312C2908523C031DD22B8A11652BA5
:1037A0008A15312C2908533C031DDA2B8A11F32B7F
:1037B0008A15312C2908543C031DE22B8A112F2C29
:1037C0008A15312C2908553C031DEA2B8A11002F3C
:1037D0008A15312C2908563C031DF22B8A113C2FE7
:1037E0008A15312C2908603C031DF82B0028312C48
:1037F0002908613C031DFE2B9D28312C2908623CC1
:10380000031D042C1029312C2908633C031D0A2CAC
:10381000C329312C2908653C031D102C492A312C61
:103820002908643C031D162CD62A312C2908663C35
:10383000031D1C2C032B312C2908673C031D222C53
:10384000242B312C2908683C031D282C4A2B312CB1
:103850002908313C031D2E2C6F2B312C8A11E72FA8
:103860008A158A150A16A22C84011F308305073099
:1038700083169F00403099002630980090308312C4
:1038800098004030831699002630980090308312BB
:1038900098004030831699002630980090308312AB
:1038A000980040308316990026309800903083129B
:1038B000980040308316990026309800903083128B
:1038C00098007130F0000230F1007C1007140714EA
:1038D000993083168700103086000B308500B53094
:1038E000831290008F018E0183160C14C030831256
:1038F0008B040F30F700073081018130840000080D
:10390000F0390738800064000008F039770480003F
:103910000A128A114B200A168A150A128A11B2203D
:103920000A168A150B138B138B1B932C83160C1002
:103930008312061564000A12942E0A167808FD00F8
:08394000FE00C72B9A2C630066
:0242000020009C
:02400E003E3F33
:00000001FF
